:10037D0004410000004C015801C1000E4873706526
:10038D006564286E2F6D696E293A0003213736009A
:10039D001C24646972656374696F6E3A637700003B
:1003AD00646972656374696F6E3A636377000140C7
:0403BD0000015601E4
:10025D00750890908506E508F07508018508897583
:10026D00571075460075470F758C10758A0F8540B0
:10027D00451204451202C2D2AFD2A9D28C12047B10
:10028D008F08E508600612049612049612047B8FFF
:10029D0008E508600B1201688F401201E512049603
:1002AD00E545B540033000D58540451204451202A1
:0502BD00C2C20080C870
:100445001204B61204D31204B61204D375903812EE
:1004550004B91204D37590011204B91204D375902E
:100465000F1204B91204D37590061204B91204D3FD
:0604750075900C0204B9B1
:1002C200E4F5097590801204B974482509F8E6FF2F
:1002D200600A1204C505091204D380EDE4F509741D
:1002E200212509F8E6FF600A1204C51204D30509A4
:1002F20080ED7590C01204B9E4F509E558B4011017
:1003020074242509F8E6FF601B1204C5050980F074
:10031200E558701074322509F8E6FF60071204C52B
:04032200050980F059
:0103260022B4
:0304B60075903806
:0C04B900C2A0C2A1C2A21204A6D2A222BC
:0E04C5008F90D2A0C2A1C2A21204A6D2A2227F
:0904D300E4FF0FEFC3946440F94B
:0104DC0022FD
:0F049600E4FFE4FE0EEEC3941E40F90FBF64F3C3
:0104A5002234
:1004A6007590FFC2A0D2A1C2A200D2A22097F122CB
:10047B007FFF908500EFF0120496E4908502F090D8
:0A048B008500E0FF6307FF53070F31
:010495002244
:10016800750900750AFE7B017A00908502E50AF0A0
:10017800908500E0FF7C005401FD700BEAC313F585
:100188000BEB13F50C803A7C00EF5402FD700AEA81
:10019800C313FEEB13240480227C00EF5404FD708B
:1001A8000AEAC313FEEB13240880107C00EF5408FE
:1001B800FD700EEAC313FEEB13240CF50CE43EF5B8
:1001C8000B74022BFBE43AFAE50A25E0F50AE50987
:0C01D80033F509430A01ED4C7090AF0CA8
:0101E40022F8
:1001E500E54024F7601324FE601624FC601A2407FA
:1001F50070657558017556F722E4F5587556012254
:10020500D200155715578006D20005570557E557F3
:10021500FAE4C39400FFE49AFE74019400FDE494AB
:1002250000FCC006C007AE46AF47AB07AA06D0071D
:10023500D006C3EF9BFBEE9AFAED9400F9EC94001F
:10024500F87F407E4B7D4C7C001203C28F448E4369
:080255008D428C4112032722A7
:10032700E4F5097B64FAF9F8AF44AE43AD42AC415A
:1003370012004AEF2430F521E47B64FAF9F8AF4460
:10034700AE43AD42AC4112004AAC00AD01AE02AFC4
:1003570003E47B0AFAF9F812004AEF2430F522E4A5
:100367007B0AFAF9F8AF44AE43AD42AC4112004AFA
:05037700EB2430F5232A
:01037C00225E
:03000B00020406E6
:10040600C0E0C083C082C0D0C28C908504E556F09F
:10041600E558700EE55625E0F556B41011755601EF
:10042600800CE556C313F556B40F037556F785577A
:0F0436008C85478AD28CD0D0D082D083D0E03250
:030000000200DC1F
:0C00DC00787FE4F6D8FD758158020123FE
:10000E0075F008758200EF2FFFEE33FECD33CDCCA9
:10001E0033CCC58233C5829BED9AEC99E58298402C
:10002E000CF582EE9BFEED9AFDEC99FC0FD5F0D609
:10003E00E4CEFBE4CDFAE4CCF9A88222B800C1B933
:10004E000059BA002DEC8BF084CFCECDFCE5F0CB71
:10005E00F97818EF2FFFEE33FEED33FDEC33FCEBAA
:10006E0033FB10D703994004EB99FB0FD8E5E4F965
:10007E00FA227818EF2FFFEE33FEED33FDEC33FC52
:10008E00C933C910D7059BE99A4007EC9BFCE99A46
:10009E00F90FD8E0E4C9FAE4CCFB2275F010EF2F8B
:1000AE00FFEE33FEED33FDCC33CCC833C810D7078B
:1000BE009BEC9AE899400AED9BFDEC9AFCE899F8C6
:0E00CE000FD5F0DAE4CDFBE4CCFAE4C8F92259
:1003C200C2D5E830E70FB2D5E4C39BFBE49AFAE466
:1003D20099F9E498F8EC30E717B2D51203F8120055
:1003E2004AE4C39BFBE49AFAE499F9E498F880039F
:1003F20012004A30D50DE4C39FFFE49EFEE49DFD4A
:04040200E49CFC2258
:1000E80002025DE493A3F8E493A34003F68001F2CF
:1000F80008DFF48029E493A3F85407240CC8C33319
:10010800C4540F4420C8834004F456800146F6DFE7
:10011800E4800B010204081020408090037DE47EF7
:10012800019360BCA3FF543F30E509541FFEE493DC
:10013800A360010ECF54C025E060A840B8E493A3A3
:10014800FAE493A3F8E493A3C8C582C8CAC583CACE
:10015800F0A3C8C582C8CAC583CADFE9DEE780BE86
:0103C100003B
:00000001FF
